:100000000B308A000B2B00000D050D052310CD329F
:10001000F4326F396F36EF33E931EB30A039F43019
:10002000EE34E332A0127310A82129103218B1194E
:10003000A03BF73BAE36EC306217633DA0060A00EA
:10004000301731000D052310C13AF437721DA0128C
:100050007310D03773366532EE34A03A7039613B95
:10006000611DA01273100D050001CA306E104334DB
:10007000F237F5397400B11A2E1A2E19B018330060
:100080002310F6327210F037F230E434200061347D
:100090006C34743469346D34653474345F3474345E
:1000A0005B34B03443345D34203461346C347434A4
:1000B00069346D34653474345F3461345B346D3469
:1000C0005D34203461346C34743469346D34653497
:1000D00074345F3470345B34503461345D342034B4
:1000E00000347334683474345F3474345B34B03443
:1000F00043345D3420347334683474345F3468348A
:100100005B34253425345D342034203441346E345E
:1001100065346D346F345B346D342F3473345D3437
:1001200063346834653463346B340D340A340D340D
:100130000A34003483168611831286110830F800C1
:10014000A1280000F817B228F813D10C031886155F
:10015000031C86117817B2287813F80BA528B0284D
:10016000000086153F308400840BB4280000F81B83
:10017000A428781BAC280800831603178C170C14CE
:10018000000000000318EB2883120C087F390313CA
:10019000CE0003170D080313CF0003170F08031336
:1001A000D0004E08D1009A204F0803178D0003138A
:1001B000500803178F0083168C170C1400000000E2
:1001C00083120313CD0BE528E82883160317EB28C9
:1001D0000A298316031783120C0D0E0D7F390313A2
:1001E000CE0003170D080313CF0003170F080313E6
:1001F000D0004E08D1009A204F0803178D0003133A
:10020000500803178F008D0A03198F0A0310031378
:10021000CD0BBC280800831603178C170C140000A4
:10022000000083120C087F3903194F290313CD00F6
:1002300003170D080313CE0003170F080313CF0095
:100240004D08D1009A204E0803178D0003134F0864
:1002500003178F0083168C170C1400000000831204
:100260000C0D0E0D7F3903194F290313CD00031711
:100270000D080313CE0003170F080313CF004D081A
:10028000D1009A204E0803178D0003134F0803175F
:100290008F008D0A03198F0A03130B290317031309
:1002A0000800831603178C170C140000000083123B
:1002B0000D080313CE0003170F080313CF00031715
:1002C0000C080313D1009A204E0803178D00031366
:1002D0004F0803178F008D0A03198F0A0313CD0BE4
:1002E00051290800043003178D0000308F000310DF
:1002F0001D300313CD00BC20203003178D000030CB
:100300008F0003130B21133003178D0000308F0073
:10031000031418300313CD00BC20223003178D00C6
:1003200000308F0003100B300313CD00BC2035309C
:1003300003178D0000308F0003130B2128300317A3
:100340008D0000308F00031412300313CD00BC2049
:100350003B3003178D0000308F0003130B2120303A
:10036000D1009A200D30D1009A200A30D1009A2075
:10037000403003178D0000308F0003130B214730EE
:1003800003178D0000308F0083168C170C140000AB
:10039000000083128C080319E4290D080313CD0013
:1003A00003170F080313CE0003170C080313D10023
:1003B0009A204D0803178D0003134E0803178F0072
:1003C0008D0A03198F0AC42971308D0000308F0007
:1003D00010300313CD0051212530D1009A208330F5
:1003E00003178D0000308F0016300313CD0051210C
:1003F0008A150A12352B0830F80000008610831683
:10040000861000008312DF0D0610031C0A2A8316D3
:100410000614831203180F2A8316061083128316FC
:1004200086148312861C122AF80BFD290000861000
:100430008316861000000614000000008614831244
:10044000861C202AF80100000618781486108316EE
:100450008610831206108316061083120800831676
:10046000061400008614000083120610831606107E
:1004700000008312861083168610C0308312DF00BE
:10048000FB212630DF00FB21B830DF00FB21831683
:100490000610000086148312861C4C2A0000502A85
:1004A00000008316061400000614000086140000E5
:1004B000831206108316061000008312861083161E
:1004C0008610C0308312DF00FB211330DF00FB21D8
:1004D0000730DF00FB21831606100000861483120C
:1004E000861C702A0000742A00008316061400007F
:1004F00006140000861400008312061083160610EE
:1005000000008312861083168610C0308312DF002D
:10051000FB212630DF00FB213930DF00FB21831671
:100520000610000086148312861C942A0000982A64
:10053000000083160614000083128A150A12392B54
:1005400052308400831300080319B32A0230F800E4
:10055000F701F70BA92AF80BA82A9730F700F70B39
:10056000AF2A800BA62A08000830E0007708E100D7
:1005700083160614000086148312861CBD2A0618F2
:100580000314061C0310F80D000083168610831256
:100590008610E00BB82A831606140000831206109A
:1005A00061080319D62A83160610831200008316E9
:1005B00086148312861CDA2A0000861083168610A1
:1005C000000083120610831606108312080083169B
:1005D000061400008614000083120610831606100D
:1005E00000008312861083168610C0308312DF004D
:1005F000FB215D08DF00FB21831606140000861432
:1006000000008312861C022B0610831606100000C1
:100610008312861083168610C1308312DF00FB21FF
:10062000F701B4227808DE00831606100000861455
:100630008312861C192B00001D2B00008316061444
:10064000000083125E08F80008008E30F7005F0893
:10065000F8005E08F900FA01F808031D392B790843
:10066000F800F9010830F702F808031D392BF701EB
:10067000412B0310F81B402BF90DF80DF703392B14
:10068000F813080062080319072CEE006608031926
:10069000072CEE02031C512B7F30EE070318072CAA
:1006A000572B8130EE02031C072C0319072C6E0810
:1006B000F700F801F901FA01ED016308EC00EC170D
:1006C0006408EB006508EA001930EE006908EA02E8
:1006D00003187A2B0130EB0203187A2BEC02031873
:1006E0007A2BED0203187A2BED0AEC0AEB0A690863
:1006F000EA07AC2B6808EB020318952B0130EC02DB
:100700000318952BED020318952BED0AEC0A6808E7
:10071000EB076908EA07031CAC2BEB0A031DAC2BA3
:10072000EC0A031DAC2BED0AAC2B67088038EC02F9
:100730000318AB2B0130ED020318AB2BED0A670851
:100740008038EC076808EB07031C892BEC0A031DB3
:10075000892BED0A892B7A14EE0BAF2BBA2B0310E1
:10076000EA0DEB0DEC0DED0D0310FA0DF90DF80D82
:10077000EF0D662B6F1CC22B0310F80CF90CFA0C52
:10078000EF0CC52BF7030319072CEF1BEE2B0310FF
:10079000EA0DEB0DEC0DED0D6908EA020318DA2BFA
:1007A0000130EB020318DA2BEC020318DA2BED020E
:1007B000031CFD2B6808EB020318E52B0130EC024B
:1007C0000318E52BED02031CFD2B67088038EC02B3
:1007D0000318EE2B0130ED02031CFD2BFA0A031D5A
:1007E000FD2BF90A031DFD2BF80A031DFD2BF70A4B
:1007F0000319072CF80CF90CFA0C6308EE006708D3
:10080000EE06EE1F052CF8170B2CF8130B2CF70136
:10081000F801F901FA01080080308318E906EE01B9
:10082000EF016508ED006908ED0664080319FC2C6A
:10083000EC00F70068080319052DEC020319A12C40
:10084000031C5F2C6908F200F2176A08F1006B08BC
:10085000F000EF010310F20CF10CF00CEF0CEC0BBC
:10086000292CED1F362C6E14192D6E106C106E167F
:100870006730840083132E2D6E12ED1B492C6C1CE7
:10088000542CF20CF10CF00CEF0CF70A0319142D98
:10089000542CF21B572C0310EF0DF00DF10DF20D3F
:1008A000F7030319142D492C6E17C12C6E1365081C
:1008B000ED00ED1F5D2CF2170D2DF2130D2D6808C4
:1008C000EC00F7006408EC026508F200F217660815
:1008D000F1006708F000EF010310F20CF10CF00CCE
:1008E000EF0CEC0B6B2CED1F782CEE14192DEE1089
:1008F0006C10EE166B30840083132E2DEE12ED1B60
:100900008B2C6C1C962CF20CF10CF00CEF0CF70AF3
:100910000319142D962CF21B992C0310EF0DF00DDA
:10092000F10DF20DF7030319142D8B2CEE17C12CCA
:10093000EE136908ED00ED1F9F2CF2170D2DF21339
:100940000D2D6908F200F2176A08F1006B08F0003B
:10095000ED1FAE2CF2136E15192D6E11EF016C10F8
:100960006730840083132E2DED1BD72C6508ED0016
:100970006C1CC12CF20CF10CF00CEF0CF70A0319F3
:10098000142DEF1FD22CF00A031DD22CF10A031DE7
:10099000D22CF20A031DD22CF20CF10CF00CF70A47
:1009A0000319142D6E1B562CEE1B982CF62C803040
:1009B000F206F21FDF2C192D6908ED00EC2C6508FA
:1009C000ED00F208031DEC2CF108031DEC2CF008DF
:1009D000031DEC2CF7010D2DF21BF62C0310EF0D6F
:1009E000F00DF10DF20DF70BEC2C142DED1FFA2C80
:1009F000F2170D2DF2130D2D6808F7006908F200AB
:100A00006A08F1006B08F0000D2D6408F700650816
:100A1000F2006608F1006708F0007208F80071083B
:100A2000F9007008FA004C2DF701F801F901FA01FC
:100A30004C2DEF01F009F109F209EF09EF0A031D4E
:100A4000272DF00A031D272DF10A0319F20A6E184B
:100A5000352CEE18772C6E19AD2CDC2C0008F00725
:100A6000031C382DF10A031D382DF20A03196C14EA
:100A700084030008F107031C402DF20A03196C14CB
:100A800084030008801F803AF20703186C146E1A62
:100A90003C2CEE1A7E2CB42C08000430DD00E7223A
:100AA0007808CD000530DD00E722780EF7000F3022
:100AB000F7057708DF01DE0025237708D6007808E0
:100AC000D7007908D8007A08D900E5007908E40051
:100AD0007808E3007708E200E901E801E7018330E4
:100AE000E60042237A08D1007908D0007808CF00C8
:100AF0007708CE00DF014D08DE00252383107A0839
:100B0000E7007908E6007808E5007708E400510876
:100B1000EB005008EA004F08E9004E08E8000C24FA
:100B20007A08D5007908D4007808D3007708D20075
:100B30005208F7005308F8005408F9005508FA0065
:100B40008A150A12452B0130DD00E722D001CF01C2
:100B5000CE017808CD000230DD00E722D20178080E
:100B6000D1000330DD00E7227808D300530DD40014
:100B7000D40DFC30D405530EF700F70CF70C0330FE
:100B8000F7057708DF01DE0025237708DE00780807
:100B9000DF007908E0007A08E100E5007908E40068
:100BA0007808E3007708E200E901E801E701813015
:100BB000E60042237A08DC007908DB007808DA00D6
:100BC0007708D900DE014D0DDF004E0DE0004F0D1E
:100BD000E100DF0DE00DE10DFC30DF05510DF90006
:100BE000520DFA00F90DFA0DFC30F9057908DE0412
:100BF0007A08DF04530EF700F70CF70C0330F70503
:100C000077085E04F7005F08F8006008F9006108E3
:100C1000FA007A08E7007908E6007808E500770826
:100C2000E400B630F700FA01F901F8016408650440
:100C300066046704031D1E2EF7012B2E0310F81BFC
:100C40002A2EE40DE50DE60DE70DFA0DF90DF80D70
:100C5000F70B1E2EF8137708DE007808DF007908FE
:100C6000E0007A08E10083107A08E7007908E600DE
:100C70007808E5007708E4005C08EB005B08EA0010
:100C80005A08E9005908E8000C247A08D8007908C5
:100C9000D7007808D6007708D5005508F700560821
:100CA000F8005708F9005808FA008A150A12502B64
:100CB00083160614000086140000831206108316A3
:100CC000061000008312861083168610C03083122F
:100CD000DF00FB212630DF00FB21B830DF00FB21E5
:100CE00083160610000086148312861C752E0000E1
:100CF000792E0000831606140000061400008614E6
:100D0000000083120610831606100000831286105E
:100D100083168610C0308312DF00FB211330DF0002
:100D2000FB210730DF00FB2183160610000086142C
:100D30008312861C992E00009D2E00008316061437
:100D400000000614000086140000831206108316AB
:100D5000061000008312861083168610C03083129E
:100D6000DF00FB212630DF00FB21B930DF00FB2153
:100D700083160610000086148312861CBD2E000008
:100D8000C12E000083160614000083128A150A1271
:100D90005B2B0130DD00E722CE017808CD00023068
:100DA000DD00E7227808CF000330DD00E722780E6F
:100DB000F7000F30F7057708DF01DE0025237708FD
:100DC000D8007808D9007908DA007A08DB00E50055
:100DD0007908E4007808E3007708E200E901E80117
:100DE000E7018330E60042237A08D3007908D20075
:100DF0007808D1007708D0004D08DA00D9015908E9
:100E00004F04F7004D08FA007708DE004D08DF00B8
:100E100025237708D9007808DA007908DB007A08FA
:100E2000DC0083107A08E7007908E6007808E5001E
:100E30007708E4005308EB005208EA005108E90083
:100E40005008E8000C247A08D7007908D600780802
:100E5000D5007708D4005408F7005508F800560864
:100E6000F9005708FA008A150A12672B5A08031965
:100E7000A62FE2005E080319A62FE2070318472FEA
:100E80007F30E202031CA62F0319A62F4B2F8130BF
:100E9000E2070318A62F6208F700F801F901FA012A
:100EA0005B08E600E6175C08E5005D08E400183022
:100EB000E200E301641C742F6108FA07031C662F2B
:100EC000F90A031D662FF80A0319E3176008F907EA
:100ED000031C6D2FF80A0319E3175F08DC00DC1709
:100EE0005C08F8070318E317E30DF80CF90CFA0C8B
:100EF000E60CE50CE40C0310E20B592F0130F70768
:100F00000318A62FF81B8B2FE60DFA0DF90DF80D1F
:100F1000F7030319A62FE61F9C2FFA0A031D9C2F27
:100F2000F90A031D9C2FF80A031D9C2FF80CF90CDD
:100F3000FA0CF70A0319A62F5B08E3005F08E30623
:100F4000E31FA42FF817AA2FF813AA2FF701F8010F
:100F5000F901FA0108002608840083132718831773
:100F60005A088000840A8001A60A0319A70A08000B
:100F700080080319CD2FCE010408CD004E10831B2D
:100F80004E140008DA00AB274D08840083134E1876
:100F90008317840A0319850AB82F8A150A12A72B0A
:100FA000CE1BE22F0F30F7004D0EF7050A30770207
:100FB0000318DD2F3030F707DF2F4E08F7077708CB
:100FC000DA00AB270F30CD050A304D020318EA2FA7
:100FD0003030EC2FCE134E08CD074D08DA00AB278A
:060FE0008A150A12A72D7C
:10100000831606140000861400008312861C06282E
:1010100006108316061000008312861083168610B1
:1010200080308312DF008A11FB218A15E330DF0054
:101030008A11FB218A15831606100000861483127C
:10104000861C2028000024280000831606140000B7
:1010500064308312D2008A11A0228A1583160614E6
:10106000000086140000831206108316061000008C
:10107000831286108316861081308312DF008A1156
:10108000FB218A150130F7008A11B4228A157808ED
:10109000CD000130F7008A11B4228A157808CE00FD
:1010A000F7018A11B4228A157808CF00831606103A
:1010B000000086148312861C5B2800005F28000055
:1010C0008316061400008312CE0CCE0C3F30CE05E2
:1010D000D3014D08D200D300D2014E0EF700F030FC
:1010E000F70577085207D0005308D1000318D10A3A
:1010F0005108DF005008DE008A1125238A15770881
:10110000D2007808D3007908D4007A08D500E50029
:101110005408E4005308E3005208E200E901FF30FC
:10112000E8007F30E7008E30E6008A1142238A15FE
:101130005230DD00B830DC002F30DB008630DA00C2
:101140007A08E1007908E0007808DF007708DE001F
:101150008A1136278A1583106630E700E600BB3017
:10116000E5008430E4007A08EB007908EA007808AA
:10117000E9007708E8008A110C248A158A150A12FA
:10118000722B8316061400008614000083120610CA
:101190008316061000008312861083168610803096
:1011A0008312DF008A11FB218A15E530DF008A11E6
:1011B000FB218A156430D2008A11A0228A15831679
:1011C00006140000861400008312861CE528061011
:1011D0008316061000008312861083168610813055
:1011E0008312DF008A11FB218A150130F7008A1172
:1011F000B4228A157808CD000130F7008A11B42294
:101200008A157808CE00F7018A11B4228A15780869
:10121000CF0083160610000086148312861C0E2948
:101220000000122900008316061400008312CE0C61
:10123000CE0C3F30CE05D3014D08D200D300D201F1
:101240004E0EF700F030F70577085207D00053082C
:10125000D1000318D10A5108DF005008DE008A11BE
:1012600025238A157708D2007808D3007908D4009E
:101270007A08D500E5007908E4007808E3007708EB
:10128000E200E901FF30E8007F30E7008E30E60041
:101290008A1142238A15DD01DC017A30DB008530BA
:1012A000DA007A08E1007908E0007808DF007708C2
:1012B000DE008A1136278A158310E701E601C03067
:1012C000E5008130E4007A08EB007908EA0078084C
:1012D000E9007708E8008A110C248A158A150A1299
:1012E0007B2BD5010408D4005510831B55144E0EDA
:1012F000F038D000D007E23ED100323ED3004E0895
:101300000F39D107D107D307E93ED200D207D20760
:101310004D0E0F39D207D307D20DD30DD309D30DFC
:101320004D080F39D307D00D0730CF000A30D3074F
:10133000D203031C9729D207D103031C9B29D10791
:10134000D003031C9F29D007CF03031CA3294F30D0
:101350008400831307305405541384075330040268
:10136000031954170008F700031DBE29541BBE299A
:10137000541AD229D419BE292030C129D4155412A7
:101380003030F707CE010408CD004E10831B4E14F9
:101390007708DA008A11AB278A154D088400831379
:1013A0004E188317840A541FAE298A150A12D62BA9
:1013B000F701F801F901FA01E201E301E401E501B5
:1013C000610860045F045E040319162A2030E600F9
:1013D0000310DA0DDB0DDC0DDD0DE20DE30DE40D88
:1013E000E50D61086502031DFF2960086402031D05
:1013F000FF295F086302031DFF295E086202031CC8
:10140000102A5E08E2025F08031C5F0FE302600817
:10141000031C600FE4026108031C610FE502031462
:10142000F70DF80DF90DFA0DE60BE829623084008E
:10143000831308000408D2005108D40003193B2A82
:101440005008DD004F08DC004E08DB004D08DA00D4
:10145000E101E0012030DF008230DE008A11362712
:101460008A157A08D0007908CF007808CE0077086E
:10147000CD00D40B202A5008DD004F08DC004E08B8
:10148000DB004D08DA005A08B63CDA00FA015B08C6
:10149000DE00DB170310DB0CDC0CDD0CFA0CF90CA6
:1014A000F80CF70CDA0B4A2ADE1F612AF709F80953
:1014B000F909FA09F70A0319F80A0319F90A0319CD
:1014C000FA0A7A08D0007908CF007808CE007708A9
:1014D000CD00D01F782AD203D216CD09CE09CF096C
:1014E000D009CD0A0319CE0A0319CF0A0319D00A6D
:1014F0003B30D9009A30D800CA30D700D6010A3024
:10150000D40051080319D20A5008DD004F08DC004E
:101510004E08DB004D08DA005908E1005808E000E9
:101520005708DF005608DE00D8210008CD00840AE5
:101530000008CE00840A0008CF00840A0008D0000A
:10154000FD308407F708031DB82A510A5402031915
:10155000B82A52080319BA2A0F3954020319B22AB9
:101560000318F22AD21BF22A521BBA2A2030EC2A84
:101570002030D205D21ECA2AD2125108031DD2032E
:101580007708D2002D30DA008A11AB278A1552086D
:10159000F700D20151085402031DDA2A7708D2005D
:1015A0002E30DA008A11AB278A155208F700203056
:1015B000D20500303030D21EEC2AD2125108031D61
:1015C000D2037708D2002D30DA008A11AB278A15B2
:1015D0005208F700D2013030F7077708DA008A1195
:1015E000AB278A155908DD005808DC005708DB00D6
:1015F0005608DA00E101E001DF010A30DE00D821FF
:101600007A08D9007908D8007808D7007708D6007A
:10161000D40B842A0800840183131F3083057130A2
:1016200083168F000F088611831286158316031701
:101630000908C039890003131F129F1200300317D5
:10164000880083128701880189010313A001A10189
:101650003030A2002E30A3003130A400A501A60135
:10166000A701BD01BC018A1172298A15CB018A111B
:101670002F2A8A150230CD00FA30D2008A11A0221A
:101680008A15CD0B3C2B8A114D2D8A157A08AB009B
:101690007908AA007808A9007708A8008A11A32D64
:1016A0008A157A08AF007908AE007808AD0077088F
:1016B000AC008A11582E8A150230CD00FA30D200C3
:1016C0008A11A0228A15CD0B5E2B8A11C92E8A158C
:1016D0007A08B3007908B2007808B1007708B00042
:1016E000CC0100287A08B7007908B6007808B50060
:1016F0007708B400C1287A08BB007908BA007808D6
:10170000B9007708B8002130F700F70B852B24309B
:10171000D1008A119A208A152130F700F70B8E2B01
:10172000A7013E30A6004D30DA008A11AB278A159A
:101730005330DA008A11AB278A155430DA008A1147
:10174000AB278A152230840083138A11B82F8A159B
:101750002030DA008A11AB278A15CA013E304A07C9
:101760008400831380080319CC2B2130F700F70B7A
:10177000B72B3E304A07840083130008CD004D0884
:10178000D1008A119A208A154A08CA0A3E3E84006E
:1017900083130008CB06AE2BA7013E30A600013014
:1017A00084003D08CE003C08CD0071292030DA00CD
:1017B0008A11AB278A15CA013E304A078400831379
:1017C00080080319FA2B2130F700F70BE52B3E3088
:1017D0004A07840083130008CD004D08D1008A1108
:1017E0009A208A154A08CA0A3E3E840083130008DC
:1017F000CB06DC2BA7013E30A600023084002B086C
:10180000D0002A08CF002908CE002808CD000230D9
:10181000D1001A222030DA008A11AB278A15CA01BA
:101820003E304A0784008313800803192E2C213090
:10183000F700F70B192C3E304A0784008313000889
:10184000CD004D08D1008A119A208A154A08CA0A8B
:101850003E3E840083130008CB06102CA7013E30C7
:10186000A600043084003308D0003208CF003108CD
:10187000CE003008CD000230D1001A222030DA002C
:101880008A11AB278A15CA013E304A0784008313A8
:1018900080080319622C2130F700F70B4D2C3E30E5
:1018A0004A07840083130008CD004D08D1008A1137
:1018B0009A208A154A08CA0A3E3E8400831300080B
:1018C000CB06442CA7013E30A600053084002F082B
:1018D000D0002E08CF002D08CE002C08CD000230FD
:1018E000D1001A222030DA008A11AB278A15CA01EA
:1018F0003E304A078400831380080319962C213058
:10190000F700F70B812C3E304A0784008313000850
:10191000CD004D08D1008A119A208A154A08CA0ABA
:101920003E3E840083130008CB06782CA7013E308E
:10193000A600043084003708D0003608CF003508F0
:10194000CE003408CD000230D1001A222030DA0057
:101950008A11AB278A15CA013E304A0784008313D7
:1019600080080319CA2C2130F700F70BB52C3E3044
:101970004A07840083130008CD004D08D1008A1166
:101980009A208A154A08CA0A3E3E8400831300083A
:10199000CB06AC2CA7013E30A600023084003B08E9
:1019A000D0003A08CF003908CE003808CD00023008
:1019B000D1001A222030DA008A11AB278A15CA0119
:1019C0003E304A078400831380080319FE2C21301F
:1019D000F700F70BE92C3E304A0784008313000818
:1019E000CD004D08D1008A119A208A154A08CA0AEA
:1019F0003E3E840083130008CB06E02CA7013E3056
:101A0000A600043084002B08D0002A08CF00290843
:101A1000CE002808CD00D1011A222030DA008A1128
:101A2000AB278A15CA013E304A0784008313800819
:101A30000319312D2130F700F70B1C2D3E304A07DA
:101A4000840083130008CD004D08D1008A119A202C
:101A50008A154A08CA0A3E3E840083130008CB0652
:101A6000132DA7013E30A600043084002B08D000BF
:101A70002A08CF002908CE002808CD000130D10067
:101A80001A222030DA008A11AB278A15CA013E30AB
:101A90004A078400831380080319652D2130F7005D
:101AA000F70B502D3E304A07840083130008CD0009
:101AB0004D08D1008A119A208A154A08CA0A3E3E6A
:101AC000840083130008CB06472DA7013E30A600F3
:101AD000023084002B08D0002A08CF002908CE004D
:101AE0002808CD000130D1001A222030DA008A11F6
:101AF000AB278A15CA013E304A0784008313800849
:101B00000319992D2130F700F70B842D3E304A0739
:101B1000840083130008CD004D08D1008A119A205B
:101B20008A154A08CA0A3E3E840083130008CB0681
:101B30007B2DA7013E30A6002A30DA008A11AB27A0
:101B40008A154B08CD003730CE008A11D02F8A1568
:101B50000D30DA008A11AB278A150A30DA008A11B3
:101B6000AB278A15CA013E304A07840083138008D8
:101B70000319CB2D2130F700F70BBC2D4A08CA0AF8
:101B80003E3E840083130008CD004D08D1008A1129
:101B90009A208A15B32D2130F700F70BCD2DBC0A02
:081BA0000319BD0A362B630096
:04400E00F52CFF3F4F
:00000001FF
